:100000000C94E0030C9408040C9408040C94080469
:100010000C9408040C9408040C9408040C94080430
:100020000C9408040C9408040C9408040C94080420
:100030000C9408040C9408040C9408040C94080410
:100040000C94D00B0C9408040C94400C0C941A0CD7
:100050000C9408040C9408040C9408040C940804F0
:100060000C9408040C9408044E414E494E495459CE
:10007000494E46CDCCCC3D0AD7233C17B7D1387773
:10008000CC2B329595E6241FB14F0A000020410089
:1000900000C84200401C4620BCBE4CCA1B0E5AAED3
:1000A000C59D742320736368616C746574206B65EF
:1000B000696E656E2041757367616E672061626568
:1000C000722069676E6F72696572742064656E2054
:1000D00045696E67616E6720616E2041352023316E
:1000E000203D204F4E202F202330203D204F4646DC
:1000F0000000000000000000000000000000000000
:1001000000000000000000000000000021206769DE
:1001100062742053656E736F72204944206D697458
:1001200020435243204665686C6572206175732ECA
:100130002045696E65205A61686C206772C3B6C33A
:100140009F65722030207A2E422028213529207385
:100150006368616C74657420C39C626572776163C7
:1001600068756E672065696E2E0000000000000053
:1001700000000000003920676962742056657273C0
:10018000696F6E20617573000000000000000000C0
:10019000000000000000000000000000000000005F
:1001A000000000000000000000000000000000004F
:1001B000000000000000000000000000000000003F
:1001C000000000000000000000000000000000002F
:1001D00000000000000000000000000000003820C7
:1001E0006769627420616C6C652054656D7065721E
:1001F00061747572656E206175732064656D20533E
:1002000070656963686572206D69742053656E73EB
:100210006F726E756D6D6572204120626973207A10
:10022000756D206C65747A74656E20566F726861A6
:100230006E64656E656E2053656E736F72206175B6
:1002400073000000000000372054656D7065726116
:10025000747572756D77616E646C756E6720616C14
:100260006C65722053656E736F72656E20616E737C
:10027000746FC39F656E0000000000000000000066
:10028000000000000000000000000000000000006E
:10029000000000000000000000000000000000005E
:1002A000000000000000000000000000000000004E
:1002B000362050696E737461747573204432206205
:1002C000697320443920756E64204130206269735F
:1002D00020413520616C7320576F726420656D700A
:1002E00066616E67656E000000000000000000009F
:1002F00000000000000000000000000000000000FE
:1003000000000000000000000000000000000000ED
:10031000000000000000000000352054656D70658D
:100320007261747572656E20696D205370656963C2
:1003300068657220616B7475616C6973696572655B
:100340006E0000000000000000000000000000003F
:10035000000000000000000000000000000000009D
:10036000000000000000000000000000000000008D
:10037000000000000000000000000000000000007D
:10038000000034204175746F6D6174697363686532
:10039000732073657269656C6C6573206175736732
:1003A0006562656E206465722054656D706572616A
:1003B000747572656E205B335D206E6163682057D3
:1003C000616E646C756E6720203431204F4E20348E
:1003D00030204F46460000000000000000000000F2
:1003E0000000000000000000000000332053656E94
:1003F000736F72656E204944206D69742054656D79
:100400007065726174757220617573676562656E7F
:1004100000000000000000000000000000000000DC
:1004200000000000000000000000000000000000CC
:1004300000000000000000000000000000000000BC
:1004400000000000000000000000000000000000AC
:1004500000000000322053656E736F72656E204994
:1004600044206D69742050696E20756E6420427559
:1004700073206175736C6573656E2E203231205365
:10048000656E736F72656E2049442065726E657586
:1004900074206175736C6573656E20737065696334
:1004A0006865726E20756E642073657269656C6C28
:1004B00020617573676562656E0000000031204140
:1004C00075746F6D617469736368657320736572A9
:1004D00069656C6C657320617573676562656E2014
:1004E0006465722054656D70657261747572656EB5
:1004F000205B385D206E6163682057616E646C75A7
:100500006E6720203131204F4E203130204F46463B
:1005100000000000000000000000000000000000DB
:10052000000000000000302045696E7374656C6C3B
:10053000756E6720646573204162667261676569E4
:100540006E74657276616C6C73207A2E422E203048
:1005500033303020496E74657276616C6C20616C4A
:100560006C65203330302053656B756E64656E208A
:1005700064656661756C7420333000000000000013
:10058000000000000000000000000000000000610A
:1005900020676962742054656D706572617475724C
:1005A00020766F6E2053656E736F7220284129206C
:1005B0006175732C206220676962742054656D70C8
:1005C00065726174757220766F6E2053656E736FFD
:1005D000722028422920617573202E2E2E207573DB
:1005E0007700000000000000000000000000000094
:1005F000000000000000000041203D2053656E73A4
:100600006F7220494420766F6D20312E2053656E25
:10061000736F72202841292C2042203D2053656EA3
:10062000736F7220494420766F6D20322E205365FF
:100630006E736F7220284229202E2E2E757377201C
:1006400000000000000000000000000000000000AA
:10065000000000000000000000000000000000009A
:10066000003F2041757367616265206465722048B0
:10067000696C66652E20466F6C67656E64204DC39D
:10068000B6676C696368652045696E676162656E0F
:1006900020696E204648454D20756E746572207243
:1006A0006177000000000000000000000000000072
:1006B000000000000000000000000000000000003A
:1006C00000000000000000000000005EBCE2613F8E
:1006D000DD83C29C7E20A3FD1F41009D23BE46DB1F
:1006E00065F88C11AF32CA57E974443A5C417264C0
:1006F00075696E6F5C4E616E6F5C4E616E6F5F31DF
:100700005F776972655F32425F565F312E322E38F5
:100710002E315C4E616E6F5F315F776972655F325B
:10072000425F565F312E322E382E312E696E6F2089
:100730004A756E20203820323032362031373A3335
:10074000373A3230006106F8058F052605BD04549E
:1007500004EB0382031903B0024702DE0175010CAA
:1007600001A30000000000250028002B000000006D
:1007700000240027002A0000000000230026002992
:10078000000404040404040404020202020202033A
:100790000303030303010204081020408001020444
:1007A00008102001020408102000000008000201C7
:1007B00000000304070000000000000000009E0C81
:1007C00011241FBECFEFD8E0DEBFCDBF24E0AAEFDB
:1007D000B1E001C01D92A43FB207E1F711E0A0E033
:1007E000B1E0EEEAF2E302C005900D92AA3FB10734
:1007F000D9F713E0C0EED3E004C02197FE010E94B8
:100800005D17CF3DD107C9F70E94D40C0C94551940
:100810000C94000090E0FC01E755F84F2491FC0196
:10082000EB56F84F3491FC01EF57F84FE491EE236B
:10083000C1F1222339F02330E9F090F4213001F1A5
:10084000223011F1F0E0EE0FFF1FE958F84FA591AB
:10085000B491EC91E32381E090E029F580E00895E4
:100860002730A9F02830C9F0243061F7809180004A
:100870008F7D03C0809180008F7780938000E2CFCE
:1008800084B58F7784BDDECF84B58F7DFBCF80911B
:10089000B0008F778093B000D5CF8091B0008F7D6E
:1008A000F9CF80E090E00895CF93DF9390E0FC01D2
:1008B000EB56F84F24918F57984FFC018491882371
:1008C000C9F090E0880F991FFC01E359F84FA591FA
:1008D000B491FC01ED59F84FC591D49161110DC04F
:1008E0009FB7F8948C91209582238C93888128233C
:1008F00028839FBFDF91CF910895623051F49FB755
:10090000F8943C91822F809583238C93E8812E2B41
:10091000EFCF8FB7F894EC912E2B2C938FBFEACFAB
:100920003FB7F8948091810290918202A091830256
:10093000B091840226B5A89B05C02F3F19F00196FF
:10094000A11DB11D3FBFBA2FA92F982F8827BC0129
:10095000CD01620F711D811D911D42E0660F771F51
:10096000881F991F4A95D1F708958F929F92AF9251
:10097000BF92CF92DF92EF92FF924B015C010E94F7
:1009800090046B017C010E9490046C197D098E0912
:100990009F09683E734081059105A8F321E0821A02
:1009A0009108A108B10888EEC80E83E0D81EE11CAA
:1009B000F11C81149104A104B10429F7FF90EF9078
:1009C000DF90CF90BF90AF909F908F9008952FB7FA
:1009D000F89460917D0270917E0280917F029091E7
:1009E00080022FBF0895AF92BF92CF92DF92EF9215
:1009F000FF920F931F93CF93DF936C017B018B01C9
:100A0000040F151FEB015E01AE18BF08C017D10718
:100A100059F06991D601ED91FC910190F081E02DA2
:100A2000C6010995892B79F7C501DF91CF911F91F7
:100A30000F91FF90EF90DF90CF90BF90AF9008950F
:100A4000FC01538D448D252F30E0842F90E0821BD4
:100A5000930B541710F0CF96089501970895FC0159
:100A6000918D828D981761F0A28DAE0FBF2FB11DB1
:100A70005D968C91928D9F5F9F73928F90E0089509
:100A80008FEF9FEF0895FC01918D828D981731F0C3
:100A9000828DE80FF11D858D90E008958FEF9FEF17
:100AA0000895FC01918D228D892F90E0805C9F4FED
:100AB000821B91098F739927089585E394E00E9422
:100AC000510521E0892B09F420E0822F089580E070
:100AD00090E0892B29F00E945D0581110C940000A3
:100AE0000895FC01A48DA80FB92FB11DA35ABF4FC3
:100AF0002C91848D90E001968F739927848FA6891D
:100B0000B7892C93A089B1898C91837080648C9370
:100B1000938D848D981306C00288F389E02D80811F
:100B20008F7D80830895EF92FF920F931F93CF9351
:100B3000DF93EC0181E0888F9B8D8C8D98131AC018
:100B4000E889F989808185FF15C09FB7F894EE89FF
:100B5000FF896083E889F98980818370806480835C
:100B60009FBF81E090E0DF91CF911F910F91FF90A7
:100B7000EF900895F62E0B8D10E00F5F1F4F0F734F
:100B80001127E02E8C8D8E110CC00FB607FCFACF0A
:100B9000E889F989808185FFF5CFCE010E94710532
:100BA000F1CFEB8DEC0FFD2FF11DE35AFF4FF082DB
:100BB0009FB7F8940B8FEA89FB8980818062CFCF41
:100BC000682F85E394E00C9493056DE285E394E04F
:100BD0000C949305CF93DF93EC01888D8823B9F0B3
:100BE000AA89BB89E889F9898C9185FD03C0808138
:100BF00086FD0DC00FB607FCF7CF8C9185FFF2CFB5
:100C0000808185FFEDCFCE010E947105E9CFDF9194
:100C1000CF910895DC012C911196ED91FC91F894FF
:100C20008181822B81839281322F3095932392830D
:100C300087E090E00197F1F781818323818383E24C
:100C400090E00197F1F790817894EFECF0E0319724
:100C5000F1F7922381E009F480E00895FC0190818E
:100C60000180F281E02D292F209560FF14C0F894B7
:100C70008281822382838181892B8183A3E2B0E0F8
:100C80001197F1F78281982B9283789487ED90E009
:100C90000197F1F70895F8948281822382838181FC
:100CA000892B8183AFEFB0E01197F1F78281982B08
:100CB000928378948FE090E0EBCFEF92FF920F93C6
:100CC0001F93CF93DF93EC01E62E08E010E0FF24A2
:100CD000F39461E08E2D8F2109F460E0CE010E9433
:100CE0002E06FF0C01501109A1F7F894E981FA8151
:100CF00091818881809589238183E981FA8192811C
:100D000088818095892382837894DF91CF911F9188
:100D10000F91FF90EF900895FC0190810180F28186
:100D2000E02DF8948181292F209582238183789466
:100D30003DE743E050E0315029F1DA011197F1F736
:100D400080818923C1F3F894828182238283818107
:100D5000892B81837894ABE7B7E01197F1F7F8948A
:100D6000818182238183A3E1B1E01197F1F7808132
:100D7000982381E009F080E07894E3E6F6E031978B
:100D8000F1F7089580E00895EF92FF920F931F937B
:100D9000CF93DF9310923304DEE087E2E82EFF2446
:100DA000F394C0913304C230C8F4CD9F8001112464
:100DB0000E521B4FC8010E948C06882359F06CEC20
:100DC000C8010E945D06C7010197F1F764E4C801FC
:100DD0000E945D06CF5FC0933304E3CF0E94E70417
:100DE00060930D0170930E0180930F019093100199
:100DF00081E080938D028091890290918A02A09176
:100E00008B02B0918C028093850290938602A0930E
:100E10008702B0938802DF91CF911F910F91FF90CD
:100E2000EF9008952F923F924F925F926F927F9230
:100E30008F929F92AF92BF92CF92DF92EF92FF92EA
:100E40000F931F93CF93DF9300D000D0CDB7DEB7C1
:100E5000109234042FE0722E3EE0632E812C912CF0
:100E600040EAA42E42ECB42E5090340480918E02BD
:100E7000581608F012C1052D10E0709E9001719E69
:100E8000300D112421573D4F3A832983690138E001
:100E9000C30ED11CE981FA818085869DC001112491
:100EA0008E529B4F0E948C06E981FA81E084E69C79
:100EB0007001112497012E523B4F790165E5C9015C
:100EC0000E945D06E981FA816191FA83E983C70195
:100ED0000E945D0629813A812C153D0599F7709E87
:100EE000F001719EF00D1124E157FD4FCF010896DE
:100EF0009A8389838085869DC00111246EEB8E5272
:100F00009B4F0E945D06109233044090330498E09A
:100F10009415C0F4ABEFB1E099E0E0E0915009F432
:100F200037C08D918E27E82FEF70F0E0E653F94F30
:100F30002491E82FE295EF70F0E0E652F94FE4914A
:100F4000E227ECCFE981FA81F081F69D900111242E
:100F50002E523B4F3C832B83E42CF12C98E0C92E7E
:100F6000D12C312C222423948B819C810E940A064F
:100F700081113228220C81E0C81AD108A9F7F701A3
:100F8000E550FE4F308281E0840D80933304BDCF65
:100F9000809103028E1360C0709EF001719EF00D6F
:100FA0001124E157FD4F12868081823209F443C03B
:100FB000883209F440C0803109F06FC091E090930D
:100FC000FA016091FB017091FC018091FA01882384
:100FD000A9F183E0660F771F8A95E1F780910202FD
:100FE000803149F480910102ECE0F0E0E81BF10966
:100FF000607F6E0F7F1F709E9001719E300D1124D7
:1010000021573D4F3A832983072E000C880B990BFB
:101010000E94B21420E030E040E85DE30E94111528
:10102000E981FA81638774878587968781E0850DDA
:101030008093340419CF1092FA01C3CF8091FF013D
:10104000807611F4687FD7CF803211F46C7FD3CFD4
:10105000803489F66E7FCFCF709EF001719EF00DC7
:101060001124E157FD4F81858E3F10F48F5F8187FA
:10107000909100019923D1F2709EF001719EF00DC4
:101080001124E157FD4F82858F5F8287891770F2A7
:1010900083869486A586B686C9CF0F900F900F9051
:1010A0000F90DF91CF911F910F91FF90EF90DF9004
:1010B000CF90BF90AF909F908F907F906F905F90F8
:1010C0004F903F902F900895FC0101900020E9F788
:1010D0003197AF01481B590BBC0185E394E00C9498
:1010E000F3048F929F92AF92BF920F931F93CF936F
:1010F000DF93CDB7DEB7A1970FB6F894DEBF0FBE72
:10110000CDBF19A2423008F44AE08E010F5D1F4F97
:10111000842E912CB12CA12CA50194010E943B1787
:10112000E62FB901CA01EA30F4F4E05DD801EE938C
:101130008D01232B242B252B79F790E080E010974D
:1011400019F0CD010E946408A1960FB6F894DEBF95
:101150000FBECDBFDF91CF911F910F91BF90AF9088
:101160009F908F900895E95CE1CF89E291E00C9423
:101170006408CF93DF930E94E005EC010E94B5085C
:101180008C0F9D1FDF91CF910895CF93DF930E9425
:101190006408EC010E94B5088C0F9D1FDF91CF9170
:1011A00008950C9464082F923F924F925F926F9231
:1011B0007F928F929F92AF92BF92CF92DF92EF92E7
:1011C000FF920F931F93CF93DF93109234041092EA
:1011D00033048EE0782E9FE0492E809133048230D4
:1011E00008F0ECC0E0903304CE2CD12C7C9C800124
:1011F0007D9C100D11240E521B4FE8012D96D80135
:101200001D968C91882301F17C9CF0017D9CF00D52
:101210001124EE52FB4F13861586148680913304F9
:10122000789EF0011124EE52FB4F1386158614862A
:1012300012861186108617821682158214821382F6
:101240008F5F80933304C9CFE79C70011124F701AD
:10125000EE52FB4F7F0130903404CF010E948C0688
:10126000811108C0D8011B961C921B9718821C96EE
:101270001C92D4CF60EFC7010E945D06D1E0612CC3
:10128000512CC1E05801BBE0AB0EB11C4801ECE0B1
:101290008E0E911CC7010E940A06282EC7010E94CB
:1012A0000A06F1E02F1255C0813009F071C0C13437
:1012B00008F4AACF7C9CF0017D9CF00D1124EE5225
:1012C000FB4F5386511002C081E085877C9CF00162
:1012D0007D9CF00D1124EE52FB4F8381882309F48D
:1012E00093CF349C9001112490E080E0F901E80F45
:1012F000F91FE157FD4FD701A80FB91F13964C9165
:10130000408301968830910589F780913404489E86
:10131000F0011124E157FD4F90913304908711861D
:101320008F5F809334048C3108F45CCFDF91CF91D0
:101330001F910F91FF90EF90DF90CF90BF90AF90F3
:101340009F908F907F906F905F904F903F902F90E5
:101350000895E62DF0E0281211C0D5018C91C81730
:10136000A8F4D801AE0FBF1F13968C918D2381F482
:10137000212CC93010F4D401CC935C2EE00FF11F66
:1013800083819D2F9095892383830AC08C13F0CF8E
:10139000F801E60DF11D83818D2B83832224239494
:1013A000622DC7010E942E06CF5FDD0F11F46394FA
:1013B000D1E0B7E0B61508F06DCF79CF8091340455
:1013C00080938E02B3CFCF93DF93682F70E090E0CD
:1013D00080E04AE00E947108EC010E94B5088C0F81
:1013E0009D1FDF91CF9108954F925F926F927F92F0
:1013F0008F929F92AF92BF92CF92DF92EF92FF9225
:101400000F931F93CF936B017C01742EAC019B0152
:101410000E943617882399F08CE291E0CF911F91BA
:101420000F91FF90EF90DF90CF90BF90AF909F9083
:101430008F907F906F905F904F900C94640846015E
:101440005701E894B7F82FEF3FEF4FE75FE7C5018B
:10145000B4010E94361781110DC02FEF3FEF4FE707
:101460005FE7C501B4010E94AB1418161CF480E3B9
:1014700091E0D4CF2FEF3FEF4FE75FE4C701B60114
:101480000E94311718161CF484E391E0C7CF2FEFA8
:101490003FEF4FE75FECC701B6010E94AB1487FD39
:1014A000F3CF20E030E0A901C701B6010E94AB14E0
:1014B00010E000E087FF08C08DE20E94E0058C018B
:1014C000F7FAF094F7F8F094C0E060E070E080E0A4
:1014D0009FE37C1641F020E030E040E251E40E94BE
:1014E0009016CF5FF6CFA70196010E9424162B011C
:1014F0003C010E9402174B015C014AE00E94710806
:101500007C01E00EF11ECC23B1F1C501B4010E94B3
:10151000B0149B01AC01C301B2010E9423164B0120
:101520005C018EE20E94E005E80EF91EC15018F140
:1015300020E030E040E251E4C501B4010E94111501
:101540002B013C010E9402174B01B12CA12C4AE057
:10155000C501B4010E947108E80EF91EC501B4016D
:101560000E94B0149B01AC01C301B2010E9423167A
:101570004B015C01DBCFC701CF911F910F91FF9011
:10158000EF90DF90CF90BF90AF909F908F907F9023
:101590006F905F904F900895CF93DF93C82F82E0B4
:1015A0000E94E00510923404DFE0809134049091B1
:1015B0008E028917E8F48F5B0E94E0058CE391E0CE
:1015C0000E94D108E0913404DE9FF0011124E1571C
:1015D000FD4F638574858585968542E00E94F409F8
:1015E0000E94B508809134048F5F80933404DDCF6E
:1015F000CC2329F083E0DF91CF910C94B908DF91DF
:10160000CF91089582E00E94E00588E391E00E9476
:10161000D108609175027091760290E080E042E01E
:101620000E9471080E94B50883E00C94B908CF931A
:10163000DF93882319F082E00E94E00510923404C1
:10164000DFE09091340480918E02981708F056C024
:101650008EE391E00E94D10881E491E00E94D108DC
:101660001092330420913304283070F580913404B3
:10167000D89FC001112481579D4F820F911DFC01FD
:101680008081803120F483E491E00E94D108809130
:10169000340420913304D89FC001112481579D4FF9
:1016A000820F911DFC01608170E090E080E040E1DC
:1016B0000E947108C0913304C73010F40E94E50500
:1016C000CF5FC0933304CECF8CE391E00E94D1086A
:1016D000E0913404DE9FF0011124E157FD4F638552
:1016E00074858585968542E00E94F4090E94B508BC
:1016F000809134048F5F80933404A3CF83E0DF9123
:10170000CF910C94B9080F931F93CF93DF93EC0103
:1017100088819981009759F02A813B8126173707E4
:1017200030F081E0DF91CF911F910F9108958B01EF
:101730006F5F7F4F0E948818009759F099838883C4
:101740001B830A832C813D81232B59F7FC011082D6
:10175000E8CF80E0E7CFCF93DF93EC0162E070E069
:101760000E94830B2881398181110FC02115310519
:1017700019F0C9010E94FF17198218821D821C826C
:101780001B821A82DF91CF91089582E090E09D83C1
:101790008C8365E471E0C901DF91CF910C944E19FF
:1017A0001F920F920FB60F9211242F933F938F9396
:1017B0009F93AF93BF9380917D0290917E02A09101
:1017C0007F02B091800230917C0223E0230F2D37FD
:1017D00058F50196A11DB11D20937C0280937D02D6
:1017E00090937E02A0937F02B09380028091810249
:1017F00090918202A0918302B09184020196A11D72
:10180000B11D8093810290938202A0938302B093D2
:101810008402BF91AF919F918F913F912F910F9033
:101820000FBE0F901F90189526E8230F0296A11D5A
:10183000B11DD2CF1F920F920FB60F9211242F938A
:101840003F934F935F936F937F938F939F93AF9348
:10185000BF93EF93FF9385E394E00E947105FF919E
:10186000EF91BF91AF919F918F917F916F915F9118
:101870004F913F912F910F900FBE0F901F90189591
:101880001F920F920FB60F9211242F938F939F9355
:10189000EF93FF93E0914504F09146048081E0913D
:1018A0004B04F0914C0482FD1BC0908180914E044A
:1018B0008F5F8F7320914F04821741F0E0914E04A7
:1018C000F0E0EB5CFB4F958F80934E04FF91EF911E
:1018D0009F918F912F910F900FBE0F901F90189591
:1018E0008081F4CF1F93CF93DF93EC01162F60E03C
:1018F000812F0E945404612F70E0FB01EB56F84FDA
:10190000E491E883FB01EF57F84FE491F0E0EE0F2C
:10191000FF1FE958F84F859194919A8389831B861C
:101920001D861C861A86198618861F821E821D82B5
:101930001C821B82DF91CF911F910895E5E3F4E0B3
:101940001382128288EE93E0A0E0B0E08483958356
:10195000A683B7838BE191E09183808385EC90E04F
:101960009587848784EC90E09787868780EC90E069
:10197000918B808B81EC90E0938B828B82EC90E05A
:10198000958B848B86EC90E0978B868B118E128ED4
:10199000138E148E6BE082ED94E00E94720C6CE06A
:1019A00080EE94E00C94720CCF93DF9300D000D0C3
:1019B00000D0CDB7DEB7789484B5826084BD84B59D
:1019C000816084BD85B5826085BD85B5816085BD3A
:1019D00080916E00816080936E00109281008091F2
:1019E000810082608093810080918100816080937A
:1019F0008100809180008160809380008091B1009F
:101A000084608093B1008091B00081608093B000C9
:101A100080917A00846080937A0080917A0082605D
:101A200080937A0080917A00816080937A0080911F
:101A30007A00806880937A001092C10062E082E0B0
:101A40000E94540462E083E00E94540462E084E057
:101A50000E94540462E085E00E94540462E086E043
:101A60000E94540462E087E00E94540462E088E02F
:101A70000E94540462E089E00E94540462E08AE01B
:101A80000E94540462E08EE00E94540462E08FE001
:101A90000E94540462E080E10E94540462E081E10B
:101AA0000E94540462E082E10E94540462E083E1F7
:101AB0000E945404E0914504F091460482E0808342
:101AC000E0914104F09142041082E0914304F091CE
:101AD000440487E6808310924D04E0914904F0911C
:101AE0004A0486E08083E0914704F09148048081B5
:101AF00080618083E0914704F09148048081886090
:101B00008083E0914704F09148048081806880835D
:101B1000E0914704F091480480818F7D80836AE0E2
:101B200070E080E090E00E94B5040E94C4066AE084
:101B300070E080E090E00E94B5040E94D30810920B
:101B40008D0282E00E94E00588E491E00E94D108C5
:101B500083E00E94B9081FE048EE842E43E0942EF3
:101B6000A12CB12C50E0252E50E0352E01E065E08F
:101B700070E080E090E00E94B50420E220930C0128
:101B8000109208011092090110920A0110920B01A3
:101B90000E94E7046093890270938A0280938B020B
:101BA00090938C02C0900D01D0900E01E0900F0137
:101BB000F09010016C197D098E099F09683E7340F1
:101BC00081059105F0F080918D028823D1F08091FC
:101BD0008E028823B1F00E94120780917B02882335
:101BE00029F08091070180270E94CC0A809107018B
:101BF000882329F080917B0280270E94170B109286
:101C00008D028091890290918A02A0918B02B091FD
:101C10008C024091850250918602609187027091FA
:101C20008802841B950BA60BB70B409103015091C2
:101C30000401609105017091060184179507A607BC
:101C4000B70710F00E94C4060E94E704C090770214
:101C5000D0907802E0907902F0907A026C197D09B8
:101C60008E099F09643671058105910508F43EC10E
:101C70000E94E7042B013C010E94E704E4E6CE0E3B
:101C8000D11CE11CF11C4C0C5D1C6E1C7F1C461A07
:101C9000570A680A790A4092770250927802609255
:101CA000790270927A0282E00E940A042091750201
:101CB00030917602892B09F07CC121603093760245
:101CC0002093750283E00E940A04209175023091EE
:101CD0007602892B09F06FC122603093760220933F
:101CE000750284E00E940A04209175023091760208
:101CF000892B09F062C1246030937602209375022B
:101D000085E00E940A042091750230917602892BA9
:101D100009F055C12860309376022093750286E061
:101D20000E940A042091750230917602892B09F0F5
:101D300048C12061309376022093750287E00E94AB
:101D40000A042091750230917602892B09F03BC17B
:101D50002062309376022093750288E00E940A0484
:101D60002091750230917602892B09F02EC12064F2
:101D7000309376022093750289E00E940A04209134
:101D8000750230917602892B09F021C120683093C9
:101D90007602209375028AE00E940A04209175025F
:101DA00030917602892B09F014C1316030937602AC
:101DB000209375028EE00E940A04209175023091F2
:101DC0007602892B09F007C13260309376022093A6
:101DD00075028FE00E940A0420917502309176020C
:101DE000892B09F0FAC03460309376022093750293
:101DF00080E10E940A042091750230917602892BBD
:101E000009F0EDC03860309376022093750281E1CD
:101E10000E940A042091750230917602892B09F004
:101E2000E0C03061309376022093750282E10E9417
:101E30000A042091750230917602892B09F0D3C0F3
:101E400030623093760220937502E0907502F09034
:101E50007602809174028111F9C3E894F6F8F09249
:101E60007602E092750280917202909173029F7BDC
:101E70009093730280937202809175029091760222
:101E800090689093760280937502209101013091C1
:101E900002012838334140F01092020110920101F2
:101EA000909373028093720220910101309102019C
:101EB0002F5F3F4F3093020120930101283B3B40AD
:101EC00038F420917202309173028217930731F037
:101ED00010920201109201010E94020B8091750282
:101EE00090917602909373028093720285E394E05E
:101EF0000E945105181619060CF0C6C085E394E03F
:101F00000E942F0580930C011A8219821C821B8269
:101F10001E821D8266E070E0CE0101960E94830B56
:101F200029813A81811168C02115310519F0C90153
:101F30000E94FF171A8219821E821D821C821B8238
:101F400085E394E00E9451057C0181E0E816F104EC
:101F500059F485E394E00E942F058E3008F056C0B6
:101F6000CE0101960E94AB0BF12CE12C85E394E0AD
:101F70000E945105181619067CF485E394E00E942E
:101F80002F058E3048F090ED980F9A3008F44CC031
:101F9000CE0101960E94AB0B85E394E00E945105AF
:101FA000181619060CF055C085E394E00E942F0521
:101FB000EFCF2E7F83CE2D7F90CE2B7F9DCE277FA0
:101FC000AACE2F7EB7CE2F7DC4CE2F7BD1CE2F773A
:101FD000DECE3E7FEBCE3D7FF8CE3B7F05CF377F19
:101FE00012CF3F7E1FCF3F7D2CCF6894F6F8F09242
:101FF0007602E092750240CF86E090E09E838D836A
:102000006EE471E0C9010E944E199ACF2D813E8184
:10201000232B21F0E981FA81309721F410920702F5
:10202000E7E0F2E08083A2CF2D813E81E216F30645
:1020300020F4E981FA81309749F410920702E7E031
:10204000F2E080839FEFE91AF90A90CFEE0DFF1DB1
:10205000F8CF89819A81009709F442C00E942F131A
:102060000E940217609308017093090180930A018E
:1020700090930B0185E394E00E94EA0589819A819F
:10208000009711F00E94FF17E0910C01E152EF312F
:1020900008F0D0C20E2E000CFF0BEF5AFF4E0C942E
:1020A0005D173A121A13BF121A131A131A131A13BE
:1020B0001A131A131A131A131A131A131A131A13B8
:1020C000741015113711CA11CE11E911EC11EF116D
:1020D000F211F6111A131A131A131A131A130D12F6
:1020E00060E070E0CB01BCCF82E00E94E00520916F
:1020F00008013091090140910A0150910B012F3FD5
:10210000EFEF3E074E075E0709F060C060910301E4
:10211000709104018091050190910601A50194013F
:102120000E943B17CA01B9014AE00E94710885E587
:1021300091E00E94C508F0900C019FEBE92EEF0C96
:1021400029E12E1508F44EC282E00E94E005E092DB
:1021500034048F2D0E94E00581E491E00E94D108B3
:102160001092330420913304283008F038C2809153
:102170003404189FC001112481579D4F820F911D77
:10218000FC018081803120F483E491E00E94D10839
:102190008091340420913304189FC0011124815789
:1021A0009D4F820F911DFC01608170E090E080E006
:1021B00040E10E947108F0903304F6E0FF1510F042
:1021C0000E94E505F394F0923304CCCF2A30310518
:1021D0004105510528F1A8EEB3E00E94D2156093A5
:1021E00003017093040180930501909306016091AF
:1021F0000301709104018091050190910601A501F0
:1022000094010E943B17CA01B9014AE00E9471087B
:1022100085E591E00E94C50883E00E94B9088BCF54
:102220008FE591E00E94C508E2CF82E00E94E005C0
:102230008091080190910901A0910A01B0910B01D0
:102240000097A105B10549F410927B0280917B02B1
:10225000882351F088E791E0DDCF0197A105B10512
:10226000A9F700937B02F2CF8BE791E0D3CF809167
:10227000080190910901A0910A01B0910B01019709
:10228000A105B10511F40E94D30882E00E94E00587
:10229000109234048091340490918E02891708F0D2
:1022A00070C08F5B0E94E00581E491E00E94D1083C
:1022B0001092330420913304283078F5809134044F
:1022C000189FC001112481579D4F820F911DFC0161
:1022D0008081803120F483E491E00E94D1088091D4
:1022E000340420913304189FC001112481579D4F5D
:1022F000820F911DFC01608170E090E080E040E180
:102300000E947108F0903304F6E0FF1510F00E946F
:10231000E505F394F0923304CDCF8FE791E00E946E
:10232000D108E09134041E9FF0011124E157FD4FC4
:10233000608570E06F5F7F4F072E000C880B990B54
:102340004AE00E94710885E891E00E94D108E0917E
:1023500034041E9FF0011124E157FD4F608570E0A9
:102360006F5F7F4F072E000C880B990B4AE00E948D
:1023700071080E94B508809134048F5F8093340403
:1023800089CF8CE891E00E94D10880918E020E9452
:10239000E30942CF81E00E94170BCDCE82E00E947C
:1023A000E0058091080190910901A0910A01B09186
:1023B0000B010097A105B10529F410920701809146
:1023C000070146CF0197A105B105C9F700930701A1
:1023D000F6CF0E941207AFCE0E94020BACCE0E9435
:1023E000C406A9CE81E00E94CC0AA5CE82E00E945C
:1023F000E0053AEEE32E36E0F32EF7016491662312
:1024000049F085E394E00E949305FFEFEF1AFF0A7D
:10241000892B99F70E94B508FFCE10928D0280910A
:10242000890290918A02A0918B02B0918C028093D4
:10243000850290938602A0938702B093880282E07F
:102440000E94E00525E4E22E27E0F22EF7016591D7
:10245000749188E092E00E94331388E092E00E9439
:10246000C50822E0E20EF11C83E697E08E159F0579
:1024700069F7D2CE8091080190910901A0910A01DB
:10248000B0910B0185369105A105B10510F480933B
:10249000000182E00E94B908109234049091340443
:1024A00080918E02981708F063C08EE391E00E943D
:1024B000D10881E491E00E94D10810923304209168
:1024C0003304283078F580913404189FC00111241A
:1024D00081579D4F820F911DFC018081803120F436
:1024E00083E491E00E94D108809134042091330468
:1024F000189FC001112481579D4F820F911DFC012F
:10250000608170E090E080E040E10E947108F0900E
:102510003304F6E0FF1510F00E94E505F394F09205
:102520003304CDCF8EE991E00E94D108E0913404CC
:102530001E9FF0011124E157FD4F618570E090E08E
:1025400080E04AE00E9471088BEA91E00E94D10885
:10255000E09134041E9FF0011124E157FD4F828564
:102560000E94E309809134048F5F8093340496CFF6
:1025700081EB91E00E94D1088091000108CF409149
:1025800008015091090160910A0170910B014230DC
:1025900051056105710508F0CECD842F81708093BF
:1025A00074022091750230917602809172029091AE
:1025B0007302452B462B472B59F03064309376023B
:1025C0002093750290649093730280937202B3CD4E
:1025D0003F7B30937602209375029F7BF4CF83E09C
:1025E0000E94B908F0900C018FE9E82EEF0C29E168
:1025F0002E1500F182E00E94E005E092340480EEA6
:102600008F0D0E94E0058CE391E00E94D108E091DB
:1026100034041E9FF0011124E157FD4F638574853A
:102620008585968542E00E94F4090E94B50883E002
:102630000E94B9082114310409F499CA0E945D0569
:10264000882309F493CA0E94000090CA83E10E9483
:102650000A04892B09F4C9CCE894F6F8C8CC66279B
:1026600077270C943A13FB01DC0105900D920020B2
:10267000E1F70895B0E0A0E0E0E4F3E10C94E315A5
:102680005C017B016115710519F0DB018D939C9351
:1026900085010F5F1F4FF501D0818D2F90E00E94C3
:1026A0008A146C01892BB9F5DD32B9F50F5F1F4F24
:1026B000D5011196DC91C1E05801F1E0AF1AB108E3
:1026C00043E050E060E770E0C5010E949314892B5D
:1026D00069F5680182E0C80ED11C45E050E06BE668
:1026E00070E0C6010E949314892B21F4680197E0E1
:1026F000C90ED11CE114F10419F0D701CD92DC927E
:1027000060E070E080E89FEFC111FFC060E070E022
:1027100080E89FE7FAC05801BBCFDB3229F485017E
:102720000E5F1F4FF501D181C0E0C6CF43E050E0FE
:1027300068E670E0C5010E949314892BE9F0F80166
:1027400010E000E020E030E0A9015F01B0ED8B2E49
:102750008D0E89E08815C8F19C2E689491F88C2F15
:102760008870C2FF16C0811102C00F5F1F4F3196E3
:10277000D501DC91C92DE9CFE114F10429F00E5FF8
:102780001F4FF7011183008360E070E080EC9FE74A
:10279000BCC0882311F001501109A5E0B0E00E94EF
:1027A000D2159B01AC01220F331F441F551F280D6A
:1027B000311D411D511D283999E93907490799E112
:1027C0005907A8F2C6609C2ED2CFAEEF8A1206C07F
:1027D000C3FD3CC09C2E689493F8C9CFDF7DD534EF
:1027E000A9F580818D3239F4C061DF0112968181B3
:1027F00062E070E006C0DF018B32C1F3119661E048
:1028000070E080535D01A61AB70A8A30F8F4E0E858
:10281000CE16ECE0DE065CF4B601660F771F660F9D
:10282000771FC60ED71ECC0CDD1CC80ED11C5D0157
:10283000FFEFAF1ABF0A8C9180538A30A8F1C4FF12
:1028400003C0D194C194D1080C0D1D1DC1FF09C056
:10285000E114F10431F081E0A81AB108D701AD927A
:10286000BC92CA01B9010E94B014C370C33009F40C
:1028700090584B015C0120E030E0A9010E94AB14AC
:10288000882309F440C0CFE9D0E017FF05C01195B7
:1028900001951109C7E8D0E06E01B8E1CB1AD10863
:1028A00080E2E82EF12C0FC0D501B1CFFE012591B9
:1028B0003591459154910E191F09C501B4010E942B
:1028C00011154B015C01D501C4010E151F0574F7EC
:1028D0002497F594E794CC16DD06A9F78A2F880F84
:1028E0008B2F881F8F3F49F020E030E0A901C50100
:1028F000B4010E94AB14811106C082E290E0909373
:10290000EF048093EE04C501B401CDB7DEB7ECE06F
:102910000C94FF1591110C947E15803219F089509A
:102920008550C8F70895FB01DC014150504088F004
:102930008D9181341CF08B350CF4805E659161348F
:102940001CF06B350CF4605E861B611171F3990B02
:102950000895881BFCCF0E94ED1408F481E00895CF
:10296000E89409C097FB3EF4909580957095619529
:102970007F4F8F4F9F4F9923A9F0F92F96E9BB27DF
:102980009395F695879577956795B795F111F8CF5B
:10299000FAF4BB0F11F460FF1BC06F5F7F4F8F4FC6
:1029A0009F4F16C0882311F096E911C0772321F0BC
:1029B0009EE8872F762F05C0662371F096E8862F54
:1029C00070E060E02AF09A95660F771F881FDAF7AB
:1029D000880F9695879597F90895990F0008550FD8
:1029E000AA0BE0E8FEEF16161706E807F907C0F095
:1029F00012161306E407F50798F0621B730B840B9D
:102A0000950B39F40A2661F0232B242B252B21F476
:102A100008950A2609F4A140A6958FEF811D811D16
:102A200008950E9424150C9498150E948A1538F078
:102A30000E94911520F0952311F00C9481150C94AF
:102A4000871511240C94CC150E94A91570F3959F3D
:102A5000C1F3950F50E0551F629FF001729FBB2795
:102A6000F00DB11D639FAA27F00DB11DAA1F649F31
:102A70006627B00DA11D661F829F2227B00DA11DE4
:102A8000621F739FB00DA11D621F839FA00D611D6A
:102A9000221F749F3327A00D611D231F849F600D8B
:102AA000211D822F762F6A2F11249F5750409AF0B4
:102AB000F1F088234AF0EE0FFF1FBB1F661F771F40
:102AC000881F91505040A9F79E3F510580F00C940B
:102AD00081150C94CC155F3FE4F3983ED4F38695B2
:102AE00077956795B795F795E7959F5FC1F7FE2BAB
:102AF000880F911D9695879597F9089599278827AE
:102B0000089597F99F6780E870E060E008959FEF6F
:102B100080EC089500240A94161617061806090674
:102B2000089500240A941216130614060506089543
:102B3000092E0394000C11F4882352F0BB0F40F4CB
:102B4000BF2B11F460FF04C06F5F7F4F8F4F9F4F0B
:102B5000089557FD9058440F551F59F05F3F71F08D
:102B60004795880F97FB991F61F09F3F79F08795F4
:102B70000895121613061406551FF2CF4695F1DF7D
:102B800008C0161617061806991FF1CF869571050D
:102B9000610508940895E894BB2766277727CB0141
:102BA00097F908950E941416A59F900DB49F900D5B
:102BB000A49F800D911D112408952F923F924F9252
:102BC0005F926F927F928F929F92AF92BF92CF92BD
:102BD000DF92EF92FF920F931F93CF93DF93CDB7C6
:102BE000DEB7CA1BDB0B0FB6F894DEBF0FBECDBF3E
:102BF00009942A88398848885F846E847D848C840F
:102C00009B84AA84B984C884DF80EE80FD800C8117
:102C10001B81AA81B981CE0FD11D0FB6F894DEBFFA
:102C20000FBECDBFED010895A29FB001B39FC001BB
:102C3000A39F700D811D1124911DB29F700D811DE8
:102C40001124911D08955058BB27AA270E943B16B6
:102C50000C9498150E948A1538F00E94911520F066
:102C600039F49F3F19F426F40C9487150EF4E0957F
:102C7000E7FB0C948115E92F0E94A91558F3BA17A8
:102C8000620773078407950720F079F4A6F50C9482
:102C9000CB150EF4E0950B2EBA2FA02D0B01B90128
:102CA00090010C01CA01A0011124FF27591B99F0C2
:102CB000593F50F4503E68F11A16F040A22F232FCE
:102CC000342F4427585FF3CF469537952795A7951E
:102CD000F0405395C9F77EF41F16BA0B620B730BC5
:102CE000840BBAF09150A1F0FF0FBB1F661F771F36
:102CF000881FC2F70EC0BA0F621F731F841F48F4EB
:102D0000879577956795B795F7959E3F08F0B0CF73
:102D10009395880F08F09927EE0F9795879508955A
:102D20000E94A4160C9498150E94911558F00E94C8
:102D30008A1540F029F45F3F29F00C948115511158
:102D40000C94CC150C9487150E94A91568F399234F
:102D5000B1F3552391F3951B550BBB27AA27621797
:102D60007307840738F09F5F5F4F220F331F441FA4
:102D7000AA1FA9F335D00E2E3AF0E0E832D09150D8
:102D80005040E695001CCAF72BD0FE2F29D0660FC5
:102D9000771F881FBB1F261737074807AB07B0E808
:102DA00009F0BB0B802DBF01FF2793585F4F3AF00E
:102DB0009E3F510578F00C9481150C94CC155F3F23
:102DC000E4F3983ED4F3869577956795B795F79594
:102DD0009F5FC9F7880F911D9695879597F908957C
:102DE000E1E0660F771F881FBB1F62177307840718
:102DF000BA0720F0621B730B840BBA0BEE1F88F727
:102E0000E09508950E94B11588F09F5798F0B92F6A
:102E10009927B751B0F0E1F0660F771F881F991F0F
:102E20001AF0BA95C9F714C0B13091F00E94CB15D1
:102E3000B1E008950C94CB15672F782F8827B85FE1
:102E400039F0B93FCCF3869577956795B395D9F767
:102E50003EF490958095709561957F4F8F4F9F4F71
:102E600008950E94ED1408F48FEF08950E94ED1468
:102E7000880B990B0895A1E21A2EAA1BBB1BFD011A
:102E80000DC0AA1FBB1FEE1FFF1FA217B307E40749
:102E9000F50720F0A21BB30BE40BF50B661F771FA1
:102EA000881F991F1A9469F7609570958095909581
:102EB0009B01AC01BD01CF010895EE0FFF1F0590EE
:102EC000F491E02D09940F931F93CF93DF938230F9
:102ED000910510F482E090E0E091F204F091F304A7
:102EE00030E020E0B0E0A0E0309799F42115310502
:102EF00009F44AC0281B390B24303105D8F58A81E2
:102F00009B816115710589F1FB0193838283FE0129
:102F100011C0408151810281138148175907E0F0A7
:102F20004817590799F4109761F012960C9312976D
:102F300013961C933296CF01DF91CF911F910F9181
:102F400008950093F2041093F304F4CF2115310592
:102F500051F04217530738F0A901DB019A01BD0176
:102F6000DF01F801C1CFEF01F9CF9093F304809313
:102F7000F204CDCFFE01E20FF31F81939193225013
:102F8000310939832883D7CF2091F0043091F1049F
:102F9000232B41F420911301309114013093F1045B
:102FA0002093F00420911101309112012115310577
:102FB00041F42DB73EB74091150150911601241BE5
:102FC000350BE091F004F091F104E217F307A0F45F
:102FD0002E1B3F0B2817390778F0AC014E5F5F4F6F
:102FE0002417350748F04E0F5F1F5093F1044093AC
:102FF000F004819391939FCFF0E0E0E09CCFCF93DA
:10300000DF930097E9F0FC01329713821282A091BE
:10301000F204B091F304ED0130E020E01097A1F448
:1030200020813181820F931F2091F0043091F104AF
:103030002817390709F061C0F093F104E093F00418
:10304000DF91CF910895EA01CE17DF07E8F54A81B5
:103050005B819E0141155105B1F7E901FB83EA83CC
:1030600049915991C40FD51FEC17FD0761F4808178
:1030700091810296840F951FE9019983888382814B
:1030800093819B838A83F0E0E0E012968D919C917E
:1030900013970097B9F52D913C911197CD010296A8
:1030A000820F931F2091F0043091F1042817390703
:1030B00039F6309751F51092F3041092F204B09360
:1030C000F104A093F004BCCFD383C283408151812B
:1030D000840F951FC817D90761F44E5F5F4F888131
:1030E0009981480F591F518340838A819B81938323
:1030F00082832115310509F0B0CFF093F304E093FA
:10310000F2049ECFFD01DC01C0CF13821282D7CF23
:10311000B0E0A0E0EEE8F8E10C94DF158C01009738
:1031200051F4CB010E9463178C01C801CDB7DEB703
:10313000E0E10C94FB15FC01E60FF71F9C01225007
:103140003109E217F30708F49DC0D901CD91DC9154
:103150001197C617D70798F0C530D10530F3CE01C7
:1031600004978617970708F3C61BD70B2297C193BE
:10317000D1936D937C93CF010E94FF17D6CF5B0153
:10318000AC1ABD0A4C018C0E9D1EA091F204B091A8
:10319000F304512C412CF12CE12C109731F5809146
:1031A000F0049091F1048815990509F05CC0461669
:1031B000570608F058C080911101909112010097B4
:1031C00041F48DB79EB74091150150911601841BB3
:1031D000950BE817F90708F055C0F093F104E09358
:1031E000F004F90171836083A0CF8D919C911197B8
:1031F00012966C90129713967C901397A815B905A8
:1032000059F56C0142E0C40ED11CCA14DB0420F154
:10321000AC014A195B09DA011296159780F06282B7
:10322000738251834083D9016D937C93E114F1043F
:1032300071F0D7011396FC93EE93129776CF2296F6
:103240008C0F9D1FF90191838083F301EFCFF093E1
:10325000F304E093F20469CF4816590608F42C01F0
:103260007D01D3019ACFCB010E9463177C010097A7
:1032700049F0AE01B8010E944519C8010E94FF172C
:10328000870153CF10E000E050CFFB01DC0102C00A
:1032900001900D9241505040D8F70895FB01DC0198
:0E32A00001900D920020E1F70895F894FFCF01
:1032AE000788133075000001FFFFFFFF2030750007
:1032BE00000000F4048000000000009305F30420D9
:1032CE0005EA0551052F0543050D0A006E616E00D6
:1032DE00696E66006F76660050696E733D004944F4
:1032EE00003A0030002D31005265616479002020D3
:1032FE0020202020002053656B756E64656E0031B2
:10330E00302053656B756E64656E2073696E642034
:10331E006D696E696D756D004F4E004F464600200B
:10332E0042757320002050696E203100416E7A6123
:10333E00686C2053656E736F72656E3A2000204381
:10334E0052435F676573616D747C00204352437C0A
:10335E00005365747A652054656D7065726174757D
:10336E007220617566202D38302E302062656920FE
:10337E00416E7A61686C2061756665696E616E6416
:10338E006572666F6C67656E6465204352432046B6
:0A339E0065686C6572203E3D20005A
:00000001FF
